:020000040000FA
:040000004BEF0BF0C7
:06002A00D9CFE5FFE1CF94
:10003000D9FF00C0E5FF01C0E5FF02C0E5FF03C036
:10004000E5FF04C0E5FF05C0E5FF06C0E5FF07C00A
:10005000E5FF08C0E5FF09C0E5FF0AC0E5FF020EA5
:10006000DBCF00F0030EDBCF01F0040EDBCF02F09C
:10007000050EDBCF03F0060EDBCF04F0070EDBCF5F
:1000800005F000C006F001C007F002C008F0035000
:1000900003E003500508036E270EE56E100EE56EB3
:1000A0000550E56E0450E56E31EC06F0096EF3CFB5
:1000B0000AF0040EE126300E092609C0E5FF06C04D
:1000C000E9FF07C0F3FF085057EC0BF0062AD8B041
:1000D000072AD8B0082A030603500EE12E0EE56E5B
:1000E00006C0E9FF07C0F3FF085057EC0BF0062AE3
:1000F000D8B0072AD8B0082A270EE56E100EE56E94
:100100000550E56E0450E56ED5EC05F0046EF3CFB6
:1001100005F0040EE126030EE56EE80EE56E0550CF
:10012000E56E0450E56E31EC06F0096EF3CF0AF08F
:10013000040EE126300E092609C0E5FF06C0E9FFDE
:1001400007C0F3FF085057EC0BF0062AD8B0072A77
:10015000D8B0082A030603500EE12E0EE56E06C045
:10016000E9FF07C0F3FF085057EC0BF0062AD8B0A0
:10017000072AD8B0082A030EE56EE80EE56E055092
:10018000E56E0450E56ED5EC05F0046EF3CF05F096
:10019000040EE126000EE56E640EE56E0550E56E78
:1001A0000450E56E31EC06F0096EF3CF0AF0040E50
:1001B000E126300E092609C0E5FF06C0E9FF07C0A9
:1001C000F3FF085057EC0BF0062AD8B0072AD8B036
:1001D000082A030603500EE12E0EE56E06C0E9FF65
:1001E00007C0F3FF085057EC0BF0062AD8B0072AD7
:1001F000D8B0082A000EE56E640EE56E0550E56E77
:100200000450E56ED5EC05F0046EF3CF05F0040E56
:10021000E126000EE56E0A0EE56E0550E56E04500F
:10022000E56E31EC06F0096EF3CF0AF0040EE1261C
:10023000300E092609C0E5FF06C0E9FF07C0F3FF3D
:10024000085057EC0BF0062AD8B0072AD8B0082A75
:10025000030603500EE12E0EE56E06C0E9FF07C04F
:10026000F3FF085057EC0BF0062AD8B0072AD8B095
:10027000082A000EE56E0A0EE56E0550E56E045084
:10028000E56ED5EC05F0046EF3CF05F0040EE12623
:10029000300E042604C0E5FF06C0E9FF07C0F3FFE7
:1002A000085057EC0BF0062AD8B0072AD8B0082A15
:1002B000032E09D02E0EE56E06C0E9FF07C0F3FF3E
:1002C000085057EC0BF00050040F036E000E012095
:1002D000046E000E0220056E0250800FF36E055072
:1002E000800FF35C05E10450015C02E10350005C07
:1002F00019E200C0E9FF01C0F3FF025000EC0BF06F
:10030000066E300A0FE1200EE56E00C0E9FF01C065
:10031000F3FF025057EC0BF0002AD8B0012AD8B0F6
:10032000022ADAD7E4CF0AF0E4CF09F0E4CF08F0EC
:10033000E4CF07F0E4CF06F0E4CF05F0E4CF04F01B
:10034000E4CF03F0E4CF02F0E4CF01F0E4CF00F01B
:10035000E4CFD9FF1200110E0001806F220E816FD1
:10036000330E826F440E836F620ED36E0F0E936E48
:10037000816A818E30EC0BF0BBEC09F0000EE56E6B
:10038000140EE56EA20EE56E000EE56E000EE56E33
:10039000FAEC04F0050EE126550EE56E000EE56E52
:1003A0007FEC0AF0020EE126000EE56EC7EC0AF0C3
:1003B000006EE12A0050E56E86EC06F0E12A110E8F
:1003C000E56E220EE56E000EE56EF5EC07F0030E0D
:1003D000E126000EE56E30EC08F0006EF3CF01F080
:1003E000E12A0150026E036A0250E56E86EC06F0C7
:1003F000E12A0050E56E86EC06F0E12AAA0E000123
:10040000906F000E016E900E006E800E026E010E57
:10041000E56E0250E56E0150E56E0050E56E030E8C
:10042000E56E000EE56E000EE56EA00EE56E79EC51
:1004300004F0080EE126000E016E800E006E800EA4
:10044000026E040EE56E0250E56E0150E56E00503E
:10045000E56E030EE56E000EE56E010EE56EA00E74
:10046000E56E79EC04F0080EE1260001906B000EB9
:10047000016E900E006E800E026E010EE56E02504F
:10048000E56E0150E56E0050E56E030EE56E000E60
:10049000E56E000EE56EA00EE56E4DEC03F0080E65
:1004A000E12600019051E56E86EC06F0E12A000E8F
:1004B000016E800E006E800E026E040EE56E02501C
:1004C000E56E0150E56E0050E56E030EE56E000E20
:1004D000E56E010EE56EA00EE56E4DEC03F0080E24
:1004E000E126000EE56E140EE56EAA0EE56E010E15
:1004F000E56E000EE56EFAEC04F0050EE126006AEA
:10050000040E005C13E2800E0024016E026A000EED
:10051000022201C0E9FF02C0EAFFEFCF01F0015063
:10052000E56E86EC06F0E12A002AEAD7FFD7120032
:10053000D9CFE5FFE1CFD9FF00C0E5FF01C0E5FF5E
:1005400002C0E5FF03C0E5FF04C0E5FF05C0E5FF0D
:1005500006C0E5FF07C0E5FF020EDBCF00F0030E8B
:10056000DBCF01F0040EDBCF02F0050EDBCF03F092
:10057000640EE56E03C0E5FF4EEC09F0046EE45036
:10058000E450300E042604C0E5FF00C0E9FF01C0BE
:10059000F3FF025057EC0BF00050010F046E000EF9
:1005A0000120056E000E0220066E640EE56E03C08B
:1005B000E5FFA4EC08F0036EE450E4500A0EE56E8B
:1005C00003C0E5FF4EEC09F0076EE450E450300E36
:1005D000072607C0E5FF04C0E9FF05C0F3FF06508A
:1005E00057EC0BF0042AD8B0052AD8B0062A0A0E18
:1005F000E56E03C0E5FFA4EC08F0036EE450E450A0
:10060000300E032603C0E5FF04C0E9FF05C0F3FF79
:10061000065057EC0BF00050020F036E000E012045
:10062000046E000E0220056E0250800FF36E05501E
:10063000800FF35C05E10450015C02E10350005CB3
:1006400019E200C0E9FF01C0F3FF025000EC0BF01B
:10065000066E300A0FE1200EE56E00C0E9FF01C012
:10066000F3FF025057EC0BF0002AD8B0012AD8B0A3
:10067000022ADAD7E4CF07F0E4CF06F0E4CF05F0A2
:10068000E4CF04F0E4CF03F0E4CF02F0E4CF01F0D4
:10069000E4CF00F0E4CFD9FF1200D9CFE5FFE1CFDE
:1006A000D9FF00C0E5FF01C0E5FF02C0E5FF03C0C0
:1006B000E5FF04C0E5FF05C0E5FF06C0E5FF07C094
:1006C000E5FF08C0E5FF020EDBCF00F0030EDBCF35
:1006D00001F0040EDBCF02F0050EDBCF03F0060EB7
:1006E000DBCF04F0070EDBCF05F0080EDBCF06F002
:1006F000090EDBCF07F056EC0AF003A003D0020E80
:10070000C86E02D0090EC86E92EC0BF00050E56E78
:100710003FEC0BF0E12A03A208D00250036E086AF6
:100720000350E56E3FEC0BF0E12A0150E56E3FEC23
:100730000BF0E12A8CEC0BF000800050E56E3FECF2
:100740000BF0E12A04C000F005C001F006C002F081
:1007500007C003F0020E035C16E3010EE56EA5EC84
:100760000AF0046EE12A04C0E5FF00C0E9FF01C001
:10077000F3FF025057EC0BF0002AD8B0012AD8B092
:10078000022A0306E7D703500FE0000EE56EA5EC42
:100790000AF0036EE12A03C0E5FF00C0E9FF01C0D3
:1007A000F3FF025057EC0BF086EC0BF0E86AE4CF55
:1007B00008F0E4CF07F0E4CF06F0E4CF05F0E4CF93
:1007C00004F0E4CF03F0E4CF02F0E4CF01F0E4CF93
:1007D00000F0E4CFD9FF1200D9CFE5FFE1CFD9FF78
:1007E00000C0E5FF01C0E5FF02C0E5FF03C0E5FF73
:1007F00004C0E5FF05C0E5FF06C0E5FF07C0E5FF53
:1008000008C0E5FF09C0E5FF0AC0E5FF0BC0E5FF32
:100810000CC0E5FF0DC0E5FF020EDBCF00F0030EBC
:10082000DBCF01F0040EDBCF02F0050EDBCF03F0CF
:10083000060EDBCF04F0070EDBCF05F0080EDBCF92
:1008400006F0090EDBCF07F0086A096A0A6A0B6A2C
:10085000200E0C6E0344010B0D6E010E0D160050A0
:1008600000260136023603360850082609360A36B5
:100870000B360D50D8A4088007500B5C08E10650D9
:100880000A5C05E10550095C02E10450085C09E3DB
:100890000450085E0550095A06500A5A07500B5A70
:1008A00000800C2ED7D703C0E9FF02C0F4FF01C0BF
:1008B000F3FF0050E4CF0DF0E4CF0CF0E4CF0BF0E9
:1008C000E4CF0AF0E4CF09F0E4CF08F0E4CF07F07A
:1008D000E4CF06F0E4CF05F0E4CF04F0E4CF03F07A
:1008E000E4CF02F0E4CF01F0E4CF00F0E4CFD9FF91
:1008F0001200D9CFE5FFE1CFD9FF00C0E5FF01C06D
:10090000E5FF02C0E5FF03C0E5FF04C0E5FF05C049
:10091000E5FF06C0E5FF07C0E5FF020EDBCF00F0F4
:10092000030EDBCF01F0040EDBCF02F0050EDBCFB0
:1009300003F0060EDBCF04F0070EDBCF05F0080E48
:10094000DBCF06F0090EDBCF07F056EC0AF003A070
:1009500003D0020EC86E02D0090EC86E92EC0BF0E6
:100960000050E56E3FEC0BF0E12A03A208D00250E4
:10097000006E036A0050E56E3FEC0BF0E12A015077
:10098000E56E3FEC0BF0E12A04C000F005C001F079
:1009900006C002F007C003F003C004F003060450D1
:1009A00013E000C0E9FF01C0F3FF025000EC0BF0C0
:1009B000046E002AD8B0012AD8B0022A0450E56E8D
:1009C0003FEC0BF0E12AE8D786EC0BF0E86AE4CFC5
:1009D00007F0E4CF06F0E4CF05F0E4CF04F0E4CF75
:1009E00003F0E4CF02F0E4CF01F0E4CF00F0E4CF75
:1009F000D9FF1200D9CFE5FFE1CFD9FF00C0E5FF55
:100A000001C0E5FF02C0E5FF03C0E5FF04C0E5FF4C
:100A1000020EDBCF00F0030EDBCF01F0040EDBCFC4
:100A200002F0050EDBCF03F0060EDBCF04F056EC30
:100A30000AF0090EC86E92EC0BF0C60EE56E3FECA4
:100A40000BF0E12A000EE56E3FEC0BF0E12AFE0E02
:100A5000E56E3FEC0BF0E12A0150400DF3CF01F0C1
:100A6000800E0126015000260050E56E3FEC0BF091
:100A7000E12A02C000F003C001F004C002F000C08F
:100A8000E9FF01C0F3FF025000EC0BF0036E0350CE
:100A90000BE0002AD8B0012AD8B0022A0350E56E34
:100AA0003FEC0BF0E12AEBD7FF0EE56E3FEC0BF0CD
:100AB000E12A86EC0BF0000EE56E0A0EE56E23ECE3
:100AC0000AF0020EE126E4CF04F0E4CF03F0E4CF15
:100AD00002F0E4CF01F0E4CF00F0E4CFD9FF120040
:100AE000D9CFE5FFE1CFD9FF00C0E5FF01C0E5FFA9
:100AF00002C0E5FF03C0E5FF04C0E5FF05C0E5FF58
:100B000006C0E5FF07C0E5FF08C0E5FF09C0E5FF37
:100B10000AC0E5FF0BC0E5FF020EDBCF00F000507E
:100B2000E56E30EC08F0016EF3CF02F0E12A036AC3
:100B3000046A002A002A0050E56E30EC08F0006ECE
:100B4000F3CF05F0E12A066A076A05500B6E0050E4
:100B50000A6E086A096A08500112095002120A5006
:100B600003120B50041204C0E9FF03C0F4FF02C0DB
:100B7000F3FF0150E4CF0BF0E4CF0AF0E4CF09F02B
:100B8000E4CF08F0E4CF07F0E4CF06F0E4CF05F0BF
:100B9000E4CF04F0E4CF03F0E4CF02F0E4CF01F0BF
:100BA000E4CF00F0E4CFD9FF1200D9CFE5FFE1CFC9
:100BB000D9FF00C0E5FF01C0E5FF02C0E5FF03C0AB
:100BC000E5FF04C0E5FF05C0E5FF06C0E5FF020E36
:100BD000DBCF00F0030EDBCF01F0040EDBCF02F021
:100BE000050EDBCF03F0046A056A0344010B066EB1
:100BF00006B011D00250022603360350015C02E118
:100C00000250005C04E2D8900332023204D0052A7C
:100C100005C004F0EAD70350015C02E10250005C19
:100C200004E30250005E0350015AD89003320232AE
:100C300004C005F004060550EEE101C0F3FF0050CA
:100C4000E4CF06F0E4CF05F0E4CF04F0E4CF03F006
:100C5000E4CF02F0E4CF01F0E4CF00F0E4CFD9FF1D
:100C60001200D9CFE5FFE1CFD9FF00C0E5FF01C0F9
:100C7000E5FF02C0E5FF03C0E5FF04C0E5FF05C0D6
:100C8000E5FF06C0E5FF07C0E5FF020EDBCF00F081
:100C9000030EDBCF01F0040EDBCF02F0050EDBCF3D
:100CA00003F0046A056A100E066E0144010B076E1C
:100CB000010E0716005000260136045004260536A2
:100CC0000750D8A404800350055C02E10250045C84
:100CD00005E30250045E0350055A0080062EE5D756
:100CE00001C0F3FF0050E4CF07F0E4CF06F0E4CFFB
:100CF00005F0E4CF04F0E4CF03F0E4CF02F0E4CF5A
:100D000001F0E4CF00F0E4CFD9FF1200D9CFE5FF26
:100D1000E1CFD9FF00C0E5FF01C0E5FF02C0E5FF5C
:100D2000020EDBCF00F000380F0B016E300E0126F3
:100D30003A0E015C02E3070E012601500001876FA5
:100D40000F0E0014016E300E01263A0E015C02E314
:100D5000070E012601500001886F8969000E016E9F
:100D6000870E006E800E026E030EE56E0250E56E79
:100D70000150E56E0050E56E000EE56E000EE56E6A
:100D8000000EE56EC60EE56E79EC04F0080EE12665
:100D9000000EE56E0A0EE56E23EC0AF0020EE12667
:100DA000E4CF02F0E4CF01F0E4CF00F0E4CFD9FFCC
:100DB0001200D9CFE5FFE1CFD9FF00C0E5FF01C0A8
:100DC000E5FF02C0E5FF03C0E5FF04C0E5FF05C085
:100DD000E5FF06C0E5FF020EDBCF00F0030EDBCF20
:100DE00001F0040EDBCF02F0050EDBCF03F0060EA0
:100DF000DBCF04F00150056E0250066EE56E055023
:100E0000E56E0050E56EF5EC07F0030EE126002AD2
:100E1000002A0350016E0450026E036A046A0250F5
:100E2000E56E0150E56E0050E56EF5EC07F0030E3F
:100E3000E126E4CF06F0E4CF05F0E4CF04F0E4CF00
:100E400003F0E4CF02F0E4CF01F0E4CF00F0E4CF10
:100E5000D9FF1200F20EF66E160EF76E000EF86E47
:100E60000900F550056E0900F550066E055002E1C7
:100E700006503BE00900F550006E0900F550016E88
:100E80000900F550026E09000900F550E96E0900ED
:100E9000F550EA6E090009000900F550036E0900DB
:100EA000F550046E09000900F6CF07F0F7CF08F0FF
:100EB000F8CF09F000C0F6FF01C0F7FF02C0F8FF4D
:100EC000035002E1045007E00900F550EE6E0306FE
:100ED000F8E20406F9D707C0F6FF08C0F7FF09C01B
:100EE000F8FF0506C4E20606C5D71200D9CFE5FF14
:100EF000E1CFD9FF00C0E5FF01C0E5FF02C0E5FF7B
:100F000003C0E5FF04C0E5FF05C0E5FF020EDBCF2F
:100F100000F0030EDBCF01F0040EDBCF02F0050E74
:100F2000DBCF03F0046A0350045C14E200C0E9FF65
:100F300001C0F3FF025000EC0BF0056E002AD8B0A0
:100F4000012AD8B0022A0550E56EEEEC0AF0E12A3B
:100F5000042AE9D7E4CF05F0E4CF04F0E4CF03F0AE
:100F6000E4CF02F0E4CF01F0E4CF00F0E4CFD9FF0A
:100F70001200D9CFE5FFE1CFD9FF00C0E5FF01C0E6
:100F8000E5FF02C0E5FF020EDBCF00F000500001DC
:100F90008A6F8B69000E016E8A0E006E800E026EE3
:100FA000020EE56E0250E56E0150E56E0050E56EF2
:100FB000000EE56E000EE56E000EE56EC60EE56EE7
:100FC00079EC04F0080EE126000EE56E0A0EE56EDF
:100FD00023EC0AF0020EE126E4CF02F0E4CF01F0A8
:100FE000E4CF00F0E4CFD9FF1200D9CFE5FFE1CF85
:100FF000D9FF00C0E5FF01C0E5FF02C0E5FF020E1A
:10100000DBCF00F0030EDBCF01F0040EDBCF02F0EC
:10101000A69EA69CA684F29E00C0A9FF0150A86EC1
:10102000550EA76EAA0EA76EA682A6B2FED70028FE
:10103000A96E0250016E026A0150A86E550EA76E8D
:10104000AA0EA76EA682A6B2FED7A694F28EE4CF11
:1010500002F0E4CF01F0E4CF00F0E4CFD9FF1200BA
:10106000D9CFE5FFE1CFD9FF00C0E5FF01C0E5FF23
:1010700002C0E5FF03C0E5FF04C0E5FF05C0E5FFD2
:10108000020EDBCF00F0A69CA69E00C0A9FFA680A2
:10109000A8CF01F0026A0028A96EA680A8CF00F0B0
:1010A000036A0050056E046A0450011205500212D2
:1010B00002C0F3FF0150E4CF05F0E4CF04F0E4CF29
:1010C00003F0E4CF02F0E4CF01F0E4CF00F0E4CF8E
:1010D000D9FF1200D9CFE5FFE1CFD9FF00C0E5FF6E
:1010E00001C0E5FF02C0E5FF03C0E5FF020EDBCF54
:1010F00000F0030EDBCF01F0040EDBCF02F000C0E6
:10110000E9FF01C0F3FF025000EC0BF0036E035047
:1011100010E0ACA2FED700C0E9FF01C0F3FF02500F
:1011200000EC0BF0AD6E002AD8B0012AD8B0022A2C
:10113000E6D7E4CF03F0E4CF02F0E4CF01F0E4CF50
:1011400000F0E4CFD9FF1200D9CFE5FFE1CFD9FFFE
:1011500000C0E5FF01C0E5FF02C0E5FF03C0E5FFF9
:10116000020EDBCF00F0030EDBCF01F0026A036A50
:1011700001BE0CD0D89001360150005C03E2D8903B
:10118000013204D0032A03C002F0F2D70150005C00
:1011900002E30150005ED890013202C003F0020663
:1011A0000350F4E10050E4CF03F0E4CF02F0E4CFC9
:1011B00001F0E4CF00F0E4CFD9FF120000C0E5FF5A
:1011C00001C0E5FF02C0E5FF03C0E5FF85EC09F0C3
:1011D000006EF3CF01F0F4CF02F0E9CF03F0000E80
:1011E000E56E0F0EE56E420EE56E400EE56E0350A5
:1011F000E56E0250E56E0150E56E0050E56EECECD8
:1012000003F0006EF3CF01F0F4CF02F0E9CF03F06A
:10121000080EE12601C0F3FF0050E4CF03F0E4CF55
:1012200002F0E4CF01F0E4CF00F0120000C0E5FFCF
:1012300001C0E5FF02C0E5FF03C0E5FF85EC09F052
:10124000006EF3CF01F0F4CF02F0E9CF03F0000E0F
:10125000E56E000EE56E030EE56EE80EE56E0350DA
:10126000E56E0250E56E0150E56E0050E56EECEC67
:1012700003F0006EF3CF01F0F4CF02F0E9CF03F0FA
:10128000080EE12601C0F3FF0050E4CF03F0E4CFE5
:1012900002F0E4CF01F0E4CF00F01200D9CFE5FF77
:1012A000E1CFD9FF00C0E5FF01C0E5FF02C0E5FFC7
:1012B00003C0E5FF04C0E5FF020EDBCF00F0030E24
:1012C000DBCF01F0026A080E036E800E0014046E7C
:1012D000D8900036D89002360450D8A4028001502D
:1012E000025C03E30150025E0080032EEED7005043
:1012F000E4CF04F0E4CF03F0E4CF02F0E4CF01F058
:10130000E4CF00F0E4CFD9FF120000C0E5FF01C038
:10131000E5FF02C0E5FF03C0E5FF04C0E5FF05C02F
:10132000E5FFB2CF00F0B3CF01F08CC002F08DC06A
:1013300003F0B2CF04F0B3CF05F00150055C02E139
:101340000050045C04E28CC002F08DC003F003C0C6
:10135000E9FF02C0F4FF05C0F3FF0450E4CF05F03D
:10136000E4CF04F0E4CF03F0E4CF02F0E4CF01F0E7
:10137000E4CF00F0120000C0E5FF01C0E5FF02C0AD
:10138000E5FFFE0E0001846F010E856F8669000E79
:10139000016E840E006E800E026E030EE56E02502A
:1013A000E56E0150E56E0050E56E000EE56E000E34
:1013B000E56E000EE56EC60EE56E79EC04F0080EE3
:1013C000E126000EE56E0A0EE56E23EC0AF0020E31
:1013D000E126E4CF02F0E4CF01F0E4CF00F0120008
:1013E000D9CFE5FFE1CFD9FF00C0E5FF01C0E5FFA0
:1013F00002C0E5FF03C0E5FF020EDBCF00F00044B2
:10140000E844FC0B016E030E0110C26EC2B2FED79F
:10141000C4CF00F0016A0050036E026AC3CF00F02F
:10142000016A005002260150032203C0F3FF02505C
:10143000E4CF03F0E4CF02F0E4CF01F0E4CF00F01A
:10144000E4CFD9FF1200D9CFE5FFE1CFD9FF00C02B
:10145000E5FF01C0E5FF02C0E5FF03C0E5FF020EA6
:10146000DBCF00F0030EDBCF01F000C002F001C0C3
:1014700003F0FF0E0026D8A001060250031006E07C
:10148000FA0E026E0000022EFDD7EFD7E4CF03F074
:10149000E4CF02F0E4CF01F0E4CF00F0E4CFD9FFD5
:1014A000120054657374696E6700000000C0E5FFA8
:1014B00001C0E5FF02C0E5FFFF0E006E1F0EC51460
:1014C000016E026AC7B4022A02500112015003E001
:1014D00000060050F3E100C001F00050D8B411EC58
:1014E0000BF00150D880E866D890016A01360150AF
:1014F000E4CF02F0E4CF01F0E4CF00F01200D9CF46
:10150000E5FFE1CFD9FF00C0E5FF01C0E5FF020E16
:10151000DBCF00F0030EDBCF01F0A69EA69CA684D5
:10152000F29E01C0A8FF00C0A9FF550EA76EAA0E2B
:10153000A76EA682A6B2FED7A694F28EE4CF01F0E3
:10154000E4CF00F0E4CFD9FF1200D9CFE5FFE1CF1F
:10155000D9FF00C0E5FF01C0E5FF020EDBCF00F0C0
:1015600056EC0AF0C58656EC0AF0C9CF01F056ECED
:101570000AF0005002E0C59A01D0C58AC588015022
:10158000E4CF01F0E4CF00F0E4CFD9FF1200D9CFCF
:10159000E5FFE1CFD9FF00C0E5FF020EDBCF00F091
:1015A000A69CA69E00C0A9FFA680A850E4CF00F08C
:1015B000E4CFD9FF120000C0E5FF01C0E5FF1F0E18
:1015C000C514006E016AC7B4012A01500012005010
:1015D000F6E1E4CF01F0E4CF00F01200D9CFE5FF4F
:1015E000E1CFD9FF00C0E5FF020EDBCF00F0ACA2D7
:1015F000FED700C0ADFFE4CF00F0E4CFD9FF12006A
:10160000E8AE04D0F3CFEAFFEE501200E8BC08D0F9
:10161000E9CFF6FFF3CFF7FFF86E0900F55012009F
:101620001200818AC69A9496828682B803D08296E6
:101630008286FBD794988298828894869488C68AFA
:101640001200200EAC6E900EAB6E0C0EAF6E000E44
:10165000E56E010EE56E23EC0AF0020EE1261200A3
:101660003F0EC716280EC66EC56A090EC86E948650
:1016700094889E96A19611EC0BF0819A1200D9CF16
:10168000E5FFE1CFD9FF020EDBCFC9FF56EC0AF030
:10169000E4CFD9FF120012EEFFF022EEFFF0F86A5D
:1016A000A68EA69C2AEC07F0ABEC01F0FFD7E8AEC3
:1016B00005D0F3CFEAFFE4CFEEFF1200E8AC120052
:1016C000120000C0E5FF006A9EBA002A0050E4CF75
:1016D00000F01200810EB16EB36AB26A00018C6B29
:1016E0008D6B1200010EC26E050EC16E940EC06E9F
:1016F00012000100421700009100000001000000EC
:10170000B36AB26A00018C6B8D6B120056EC0AF062
:10171000C584C5B4FED7120056EC0AF0C582C5B226
:10172000FED7120056EC0AF0C580C5B0FED71200F5
:1017300000018C2B01E38D2B12009EAAFED7AE5028
:041740001200000093
:00000001FF
